S00C00006D61696E2E7372656373
S113000012C02AC029C028C027C026C025C024C0C9
S113001023C022C021C020C01FC01EC01DC01CC0E0
S11300201BC01AC019C011241FBECFEDCDBF10E0F4
S1130030A0E6B0E0ECE2F1E003C0C89531960D9281
S1130040A036B107D1F710E0A0E6B0E001C01D92E0
S1130050A036B107E1F730C0D3CFCF93DF93CDB74C
S1130060DEB724970FB6F894DEBF0FBECDBF80E88D
S113007096E9A8E9B0E089839A83AB83BC8389813C
S11300809A81AB81BC810097A105B10561F089819A
S11300909A81AB81BC810197A109B10989839A83B3
S11300A0AB83BC83ECCF24960FB6F894DEBF0FBEAF
S11300B0CDBFDF91CF910895CBEDD0E0DEBFCDBFB2
S11300C08FE18093370019821A821B821C828981F6
S11300D09A81AB81BC8188309105A105B10598F75F
S11300E089819A81AB81BC81880F991FAA1FBB1F8C
S11300F0880F991FAA1FBB1F809338008091380076
S1130100816080933800A9DF9EEF809138008923B5
S11301108093380089819A81AB81BC810196A11DAD
S10F0120B11D89839A83AB83BC83D1CFCB
S9030000FC
